 pwmsdk

 Timestamp is 4fb04cc7 (Mon May 14 12:07:35 2012)

 Preferred load address is 10000000

 Start         Length     Name                   Class
 0001:00000000 00000004H .CRT$XCA                CODE
 0001:00000004 00000004H .CRT$XCZ                CODE
 0001:00000008 00000004H .CRT$XIA                CODE
 0001:0000000c 00000004H .CRT$XIZ                CODE
 0001:00000010 00000004H .CRT$XPA                CODE
 0001:00000014 00000004H .CRT$XPZ                CODE
 0001:00000018 00000004H .CRT$XTA                CODE
 0001:0000001c 00000004H .CRT$XTZ                CODE
 0001:00000020 0000002aH .rdata                  CODE
 0001:0000004c 00000023H .rdata$debug            CODE
 0001:00000070 000008f8H .text                   CODE
 0001:00000968 00000018H .xdata                  CODE
 0001:00000980 00000014H .idata$2                CODE
 0001:00000994 00000014H .idata$3                CODE
 0001:000009a8 00000048H .idata$4                CODE
 0001:000009f0 0000000cH .idata$6                CODE
 0001:00000a00 000000c7H .edata                  CODE
 0002:00000000 00000048H .idata$5                DATA
 0002:00000048 0000045cH .data                   DATA
 0002:000004a8 00000018H .bss                    DATA
 0003:00000000 000000a0H .pdata                  DATA

  Address         Publics by Value              Rva+Base       Lib:Object

 0000:00000000       ___safe_se_handler_count   00000000     <absolute>
 0000:00000000       ___safe_se_handler_table   00000000     <absolute>
 0001:00000000       __xc_a                     10001000     corelib0:crt0init.obj
 0001:00000004       __xc_z                     10001004     corelib0:crt0init.obj
 0001:00000008       __xi_a                     10001008     corelib0:crt0init.obj
 0001:0000000c       __xi_z                     1000100c     corelib0:crt0init.obj
 0001:00000010       __xp_a                     10001010     corelib0:crt0init.obj
 0001:00000014       __xp_z                     10001014     corelib0:crt0init.obj
 0001:00000018       __xt_a                     10001018     corelib0:crt0init.obj
 0001:0000001c       __xt_z                     1000101c     corelib0:crt0init.obj
 0001:0000003c       ??_C@_1O@JHINELIN@?$AAP?$AAW?$AAM?$AA?$CF?$AAd?$AA?3?$AA?$AA@ 1000103c     pwmsdk.obj
 0001:00000070       DllMain                    10001070 f   pwmsdk.obj
 0001:00000150       PwmInit                    10001150 f   pwmsdk.obj
 0001:00000230       PwmDeinit                  10001230 f   pwmsdk.obj
 0001:00000284       PwmStartDuration           10001284 f   pwmsdk.obj
 0001:00000358       PwmStop                    10001358 f   pwmsdk.obj
 0001:000003e4       PwmReset                   100013e4 f   pwmsdk.obj
 0001:000003fc       PwmReadRegisters           100013fc f   pwmsdk.obj
 0001:0000047c       PwmStart                   1000147c f   pwmsdk.obj
 0001:00000490       DisableThreadLibraryCalls  10001490 f   coredll:COREDLL.dll
 0001:000004a0       SetLastError               100014a0 f   coredll:COREDLL.dll
 0001:000004b0       DeviceIoControl            100014b0 f   coredll:COREDLL.dll
 0001:000004c0       CloseHandle                100014c0 f   coredll:COREDLL.dll
 0001:000004d0       CreateFileW                100014d0 f   coredll:COREDLL.dll
 0001:000004e0       wsprintfW                  100014e0 f   coredll:COREDLL.dll
 0001:000004f0       WriteFile                  100014f0 f   coredll:COREDLL.dll
 0001:00000500       ReadFile                   10001500 f   coredll:COREDLL.dll
 0001:00000614       _DllMainCRTStartup         10001614 f   corelib0:pegdmain.obj
 0001:00000644       __GSHandlerCheckCommon     10001644 f   corelib0:gshandler.obj
 0001:00000680       __GSHandlerCheck           10001680 f   corelib0:gshandler.obj
 0001:000006a4       __security_init_cookie     100016a4 f   corelib0:seccinit.obj
 0001:00000700       __security_check_cookie    10001700 f   corelib0:armsecgs.obj
 0001:00000714       __gsfailure                10001714 f   corelib0:armsecgs.obj
 0001:00000854       _cexit                     10001854 f   corelib0:cexit.obj
 0001:00000870       _initterm                  10001870 f   corelib0:crt0dat.obj
 0001:000008a4       _cinit                     100018a4 f   corelib0:crt0dat.obj
 0001:000008d8       __rt_udiv                  100018d8 f   corelib1:COREDLL.dll
 0001:000008e8       _XcptFilter                100018e8 f   corelib1:COREDLL.dll
 0001:000008f8       __C_specific_handler       100018f8 f   corelib1:COREDLL.dll
 0001:00000908       __security_gen_cookie2     10001908 f   corelib1:COREDLL.dll
 0001:00000918       __report_gsfailure         10001918 f   corelib1:COREDLL.dll
 0001:00000928       free                       10001928 f   corelib1:COREDLL.dll
 0001:00000938       DeleteCriticalSection      10001938 f   coredll:COREDLL.dll
 0001:00000948       InterlockedExchange        10001948 f   coredll:COREDLL.dll
 0001:00000958       TerminateProcess           10001958 f   coredll:COREDLL.dll
 0001:00000980       __IMPORT_DESCRIPTOR_COREDLL 10001980     coredll:COREDLL.dll
 0001:00000994       __NULL_IMPORT_DESCRIPTOR   10001994     coredll:COREDLL.dll
 0002:00000000       __imp_DisableThreadLibraryCalls 10002000     coredll:COREDLL.dll
 0002:00000004       __imp_SetLastError         10002004     coredll:COREDLL.dll
 0002:00000008       __imp_DeviceIoControl      10002008     coredll:COREDLL.dll
 0002:0000000c       __imp_CloseHandle          1000200c     coredll:COREDLL.dll
 0002:00000010       __imp_CreateFileW          10002010     coredll:COREDLL.dll
 0002:00000014       __imp_wsprintfW            10002014     coredll:COREDLL.dll
 0002:00000018       __imp_WriteFile            10002018     coredll:COREDLL.dll
 0002:0000001c       __imp_ReadFile             1000201c     coredll:COREDLL.dll
 0002:00000020       __imp___rt_udiv            10002020     corelib1:COREDLL.dll
 0002:00000024       __imp__XcptFilter          10002024     corelib1:COREDLL.dll
 0002:00000028       __imp___C_specific_handler 10002028     corelib1:COREDLL.dll
 0002:0000002c       __imp___security_gen_cookie2 1000202c     corelib1:COREDLL.dll
 0002:00000030       __imp___report_gsfailure   10002030     corelib1:COREDLL.dll
 0002:00000034       __imp_free                 10002034     corelib1:COREDLL.dll
 0002:00000038       __imp_DeleteCriticalSection 10002038     coredll:COREDLL.dll
 0002:0000003c       __imp_InterlockedExchange  1000203c     coredll:COREDLL.dll
 0002:00000040       __imp_TerminateProcess     10002040     coredll:COREDLL.dll
 0002:00000044       \177COREDLL_NULL_THUNK_DATA 10002044     coredll:COREDLL.dll
 0002:00000048       ?dpCurSettings@@3U_DBGPARAM@@A 10002048     DebugZones.obj
 0002:0000049c       __security_cookie          1000249c     corelib0:seccinit.obj
 0002:000004a0       __security_cookie_complement 100024a0     corelib0:seccinit.obj
 0002:000004ac       _exitflag                  100024ac     corelib0:cexit.obj
 0002:000004b0       __onexitend                100024b0     <common>
 0002:000004b4       __onexitbegin              100024b4     <common>
 0002:000004b8       g_pcsExit                  100024b8     <common>
 0002:000004bc       _pRawDllMain               100024bc     <common>

 entry point at        0001:00000614

 Static symbols

 0001:00000088       ?CallDriver@@YAHKHPAK@Z    10001088 f   pwmsdk.obj
 0001:00000518       _DllMainCRTStartupHelper   10001518 f   corelib0:pegdmain.obj
 0001:00000758       doexit                     10001758 f   corelib0:cexit.obj
